:020000040800F2
:1000000000040220010200080302000802020008A6
:1000100002020008020200080202000802020008B0
:10002000020200080202000802020008BD250008C2
:100030000202000802020008020200080202000890
:100040000202000802020008020200080202000880
:1000500002020008020200081938000845380008AA
:10006000713800089D380008C938000802020008ED
:100070000202000802020008020200080202000850
:100080000202000802020008020200080202000840
:10009000020200080202000802020008F538000807
:1000A0000202000802020008020200080202000820
:1000B0003D360008020200080202000802020008A1
:1000C0000202000802020008020200080202000800
:1000D00002020008020200082D0F0008410F00086C
:1000E0005D3900080202000802020008020200084E
:1000F00002020008020200080202000802020008D0
:1001000002020008020200080202000802020008BF
:1001100002020008020200080202000802020008AF
:10012000020200080202000802020008020200089F
:10013000020200080202000802020008020200088F
:10014000020200080202000802020008212D000835
:10015000020200080202000802020008020200086F
:10016000020200080202000802020008020200085F
:10017000020200080202000802020008020200084F
:100180000202000802020008550F000802020008DF
:10019000020200080202000802020008020200082F
:1001A000020200080202000802020008020200081F
:1001B000020200080202000802020008020200080F
:1001C00002020008020200080202000802020008FF
:1001D00002020008020200080202000802020008EF
:1001E00002020008020200080202000802020008DF
:1001F00002020008020200080202000802020008CF
:1002000002E000F000F8FEE772B6394880F3088893
:10021000384880F3098838484EF60851CEF200017C
:10022000086040F20000CCF200004EF63471CEF2CD
:1002300000010860BFF34F8FBFF36F8F40F20000E3
:10024000C0F2F0004EF68851CEF200010860BFF314
:100250004F8FBFF36F8F4FF00000E1EE100A4EF6A4
:100260003C71CEF200010860062080F31488BFF3D1
:100270006F8F02F0E1F903F06BF94FF055301F4931
:100280001B4A91423CBF41F8040BFAE71C49194A4A
:1002900091423CBF41F8040BFAE71A491A4A1B4B3A
:1002A0009A423EBF51F8040B42F8040BF8E70020D5
:1002B0001749184A91423CBF41F8040BFAE702F093
:1002C000FFF903F0AFF9144C144DAC4203DA54F8C3
:1002D000041B8847F9E700F03FF8114C114DAC4280
:1002E00003DA54F8041B8847F9E702F0E7B9000085
:1002F0000004022000240220000000080000022068
:1003000000040220E83D00080024022050240220BE
:100310005024022088410220000200080002000848
:1003200000020008000200082DE9F04F2DED108AB0
:10033000C1F80CD0D0F80CD0BDEC108ABDE8F08F1D
:10034000002383F311882846A047002001F0FCFD1C
:1003500001F0ACFD00DFFEE770B51D4C6FF07703D8
:10036000002523706FF07F061E236570A570E57071
:1003700025716571A571E57125726672A372E572CA
:1003800000F068FC20B10E2325726672A372E5723C
:1003900002F0F4F80F4B984217D00133984241F223
:1003A000883412BF002500240125002002F0ECF85B
:1003B0000DB100F053F800F0BFFC00F095FB2046B3
:1003C00000F0E0F800F04AF8F9E700242546ECE7F1
:1003D00050240220010007B008B500F003FBA0F193
:1003E00020035842584108BD07B5054B02211B8820
:1003F000ADF8043001A800F061FB03B05DF804FB28
:100400005C3A000810B51148C3680BB101F022FE38
:100410000F4C104A0D4800234FF47A7101F0DEFDB5
:10042000236813B12368013B2360636813B16368D9
:10043000013B6360084B1B7833B9636823B9022022
:1004400000F034FC3223636010BD00BF5C24022046
:100450007429022005040008702402202DE9F041CF
:10046000414C236801337CD0404D414B2A689A426D
:1004700077D9404B9B6803F1006303F5C0339A4280
:100480006FD2002000F04CFB3B4B0220187000F0B4
:1004900003FC3A4B1A6C00221A64196E1A66196E24
:1004A000596C5A64596E5A66596E596941F0800107
:1004B0005961596921F0800159615969196941F0FF
:1004C00000511961196921F0005119611B6972B657
:1004D0002B4B1C6024682D68BFF34F8FBFF36F8FC9
:1004E000083BC3F88420BFF34F8F5A6922F480324F
:1004F0005A61BFF34F8FD3F88020C2F3C906C2F30D
:100500004E325201B70743F6E07E02EA0E08384643
:100510003146013948EA000CB1F1FF3FC3F874C21B
:1005200000F14040F5D1203A12F1200FEDD1BFF398
:100530004F8FBFF36F8FBFF34F8FBFF36F8F5A692A
:1005400022F400325A610022C3F85022BFF34F8FC9
:10055000BFF36F8F202383F31188A54684F30888A7
:100560002847BDE8F08100BF008001080480010831
:10057000FF7F01085024022070240220003802402E
:1005800008ED00E02DE9F04FB34B8246B3489C687C
:100590000022C2608FB0202282F31188C2680093CB
:1005A0000AB101F057FD0023AD4AAC484FF47A710F
:1005B00001F014FD002383F31188DFF8C0B2BAF113
:1005C000000F01D0CBF800A0A64FCBF804300025D7
:1005D0003B702E464FF0FF38012000F05DFBBAF172
:1005E000000F00F0C181DBF80030002B40F0BC812F
:1005F0000FB0BDE8F08F0220FFF7EEFE002840F0BC
:10060000AF81994B1B88ADF82430022109A800F076
:1006100055FAE1E74FF47A7000F0E4F9031E019314
:10062000EFDB0220FFF7D8FE81460028E9D0019BCE
:10063000581E0428E5D8DFE800F00310131619004F
:100640000EA8052340F8143D042100F037FA4D466A
:1006500000F068FBFFF7C8FE7FE104217E48F4E765
:1006600004218248F1E704218148EEE71C25284651
:1006700000F058FA04350990042109A800F01EFA88
:100680002C2DF4D1E3E7002EBBD0002DB9D00220F1
:10069000FFF7A2FE064610B901252E46B1E701205C
:1006A00000F03EFA0220387000F0F6FA00255FFAFA
:1006B00085F9484600F04CFA0135044618B1484621
:1006C00000F056FAF3E7012302203B7000F0DAFA5B
:1006D000009B9B689C4207D2204600F023FA013021
:1006E00040F040810434F3E700243C70CBF8044030
:1006F0003546ADE7002E84D0002D82D00220387020
:1007000000F0CAFA322000F06DF9051EC4DB15F0C6
:100710000306C1D1009A926863199342BCD8B5F51B
:10072000807FB9D8DFF84C91AE420CDA4FF47A7082
:1007300000F058F90390039B002BADDB039B06F8F8
:1007400009300136F0E7C820FFF746FE06460028CC
:10075000A2D02CB9474B4FF0FF32D3F800801A607B
:10076000444B25F003052544A3EB0409AC42BFD05C
:1007700059F80410204600F0DBF9204600F0D2F9C9
:1007800059F80430984240F0ED800434EEE702203E
:10079000FFF722FE00283FF434AF4FF0000AD146A5
:1007A000009B9B689A4537D2BAF1000F17D1B8F178
:1007B000FF3F14D0CDF824802F494B68A3B100220D
:1007C00009A8135C83EA0903DBB2013251F8233034
:1007D000042A83EA1929F4D10AF1040AE0E7504611
:1007E00000F0A0F90990E7E71A46082012F0010F7F
:1007F0004FEA52021FBF82F06D4282F4380282F447
:10080000034282F020020138F0D141F82320013365
:10081000B3F5807FE8D1D2E70EA8042140F8289DE7
:1008200000F04CF914E70EA8002340F8143D6421B1
:1008300000F010F900287FF4E4AE0220FFF7CCFDB1
:1008400000283FF4DEAE099800F0A4F90EAB43F89F
:10085000240D04211846E3E7502402205C240220E2
:1008600005040008702402205E3A00085424022087
:1008700058240220742402207425022074290220A6
:100880000EA8002340F8143D642100F0E3F800288E
:100890007FF4B7AE0220FFF79FFD00283FF4B1AE12
:1008A000099800F085F90EAB43F8200DD1E702203E
:1008B000FFF792FD00283FF4A4AE00F07FF90EABE5
:1008C00043F81C0DC5E70220FFF786FD00283FF422
:1008D00098AE09A9142000F077F981460EA80421EA
:1008E00040F8189D00F0EAF8494609A898E74FF447
:1008F0007A70FFF771FD00283FF483AEB8F1FF3F37
:1009000005D1FFF771FD354801F024FB70E6414643
:10091000002000F00DF9002000F004F98045F0D02F
:100920002F4B6FE60EA8002340F8143D642100F021
:1009300091F800287FF465AE0220FFF74DFD0028F6
:100940003FF45FAEFFF750FD41F2883001F002FB4B
:10095000099800F02FFA00F0E5F94FF0000A3BE6A5
:10096000064675E63546DBE7002000F03BF80390CD
:10097000039B002BFFF633AE012000F083F9039BAD
:10098000213B122B3FF628AE01A252F823F000BF04
:10099000F70500081506000887060008D9050008B5
:1009A000D9050008D9050008F5060008D905000892
:1009B0008F0700082708000881080008AF08000812
:1009C000D9050008C7080008D9050008EF08000885
:1009D00051060008D905000825090008A086010075
:1009E000603A00082DE9F34702AE00244FF47A750F
:1009F00006F8014D144FDFF85880454397F9003051
:100A00005A1C5FFA84F901D0A34212D158F824008D
:100A100003680122D3F820A031462B46D047012895
:100A200007D10A4B9DF8070083F8009002B0BDE89B
:100A3000F0870134042CE1D14FF4FA7001F08AFA06
:100A40004FF0FF30F2E700BF002402209829022077
:100A50006C3A00082DE9F0474FF47A75144FDFF82F
:100A6000588006464D43002497F900305A1C5FFA1F
:100A700084F901D0A34210D158F82400036804225D
:100A8000D3F820A031462B46D047042805D1094B86
:100A900083F800900020BDE8F0870134042CE3D1F6
:100AA0004FF4FA7001F056FA4FF0FF30BDE8F087CE
:100AB00000240220982902206C3A000830B4074B29
:100AC0001A78074B53F822402368DD69054B0A4624
:100AD000AC460146204630BC604700BF9829022042
:100AE0006C3A0008A0860100F8B501F06BFC094CD7
:100AF000094E0A4F2070002530682378834207D9B9
:100B000001F05AFC336805440133BD423360F3D928
:100B1000F8BD00BF992902207C290220FF7F010037
:100B200001F018BD00F1006000F5C03000687047AA
:100B300007B502AB00F1006043F8041D042219461A
:100B400000F5C03001F094FC03B05DF804FB000038
:100B5000054B1A68054B1B781344834202D9104495
:100B600001F02ABC002070477C290220992902202C
:100B700038B5074D04462868204401F025FC28B903
:100B800028682044BDE8384001F036BC38BD00BFBD
:100B90007C29022010F0030308D1B0F5806F05D83E
:100BA00000F10050A0F571200068704700207047E8
:100BB000014BC058704700BF20F4F01F014B18686C
:100BC000704700BF002004E0F0B5204B1E68204BAA
:100BD0001F885D6893F90840C6F30B02BA424FEADA
:100BE000164622D09F89BA4221D01F8BBA4206D125
:100BF00002220C2404FB02335D6893F90840B6F529
:100C0000805F16D041F201039E4208BF5A24421E63
:100C10000A44013D0B46934215D215F9016F581C49
:100C20004EB1034600F8016CF5E70022E1E701222E
:100C3000DFE74124EBE72C2582421D7001D9981C87
:100C40005C70401AF0BD1846FBE700BF002004E0CE
:100C500004240220094B5B88B3F5805F09D041F280
:100C60000102934207D10122054B03EB8203D8789E
:100C700070470022F8E70020704700BF002004E022
:100C8000643A0008022802BF024B4FF480529A6176
:100C9000704700BF00100240022802BF024B4FF015
:100CA00080529A61704700BF00100240022801BFC5
:100CB000024A536983F48053536170470010024025
:100CC00010B50023934203D0CC5CC4540133F9E740
:100CD00010BD000030B5441E14F9010F0B4660B181
:100CE00093F90050854201F1010106D11AB993F937
:100CF0000020801A30BD013AEEE7002AF7D11046F5
:100D000030BD000002460346981A13F9011B002962
:100D1000FAD1704702440346934202D003F8011B04
:100D2000FAE77047024B1A78024B1A70704700BFFF
:100D30009829022000240220F8B5184C1848194DB3
:100D4000194E174F00F04CFC2146154800F074FC7A
:100D500023681648DA6ED2F8043843F00203C2F86A
:100D6000043801F0F7F82068114900F06DFD2368A0
:100D7000DA6ED2F8043823F00203C2F804384FF4D4
:100D8000E1332B60002456F82400B84202D02946F3
:100D900000F082FB0134042CF5D1F8BD643B00085F
:100DA00020370220802902206C3A000840420F00C0
:100DB000AC3B000838B50B4B1A780B4B53F822406C
:100DC0000A4B9C4205460CD0094B002118461822BC
:100DD000FFF7A0FF056001462046BDE8384000F05F
:100DE0005BBB38BD982902206C3A000820370220EE
:100DF00080290220026843681143016003B118474B
:100E000070470000024A136843F0C0031360704744
:100E100000440040024A136843F0C0031360704767
:100E200000480040024A136843F0C0031360704753
:100E3000007800402DE9F041C66D3768F5693562EC
:100E40000446280719D015F0080F0CBF0021802197
:100E5000EA0748BF41F02001AB0748BF41F040011D
:100E6000680748BF41F48071202383F31188201D57
:100E7000FFF7C0FF002383F31188E9050AD520237B
:100E800083F311884FF40071201DFFF7B3FF002397
:100E900083F31188AA060CD5202383F31188736A83
:100EA00094F864102046194000F004FB002383F3FB
:100EB00011883B0614D5280612D5202383F3118808
:100EC00004F1380000F05CFA002822DA0821201D25
:100ED000FFF790FF27F080033360002383F311882E
:100EE00079060DD56A060BD5202383F31188E26CB1
:100EF000236D9A4201D1236C6BB9002383F31188CF
:100F0000EB0610D5A26E13696BB15069BDE8F041D4
:100F10001847B062E1E71021201D27F04007FFF7D6
:100F200069FF3760E9E7BDE8F081000008B50348D4
:100F3000FFF780FFBDE8084001F050BB9C2902206C
:100F400008B50348FFF776FFBDE8084001F046BB4F
:100F5000082A022008B50348FFF76CFFBDE80840E7
:100F600001F03CBB742A022037B52D4C2D4D204694
:100F700000F086FA009404F1140000234FF400728C
:100F8000294900F047F94FF40072009404F1380049
:100F9000264B274900F0C0F9264BE3652566264C11
:100FA0000B21262000F0C4F8204600F069FA0094D6
:100FB00004F1140000234FF40072204900F02AF9D4
:100FC0004FF40072009404F138001D4B1D4900F0ED
:100FD000A3F91D4BE36525661C4C0B21272000F06F
:100FE000A7F8204600F04CFA04F114000094002306
:100FF0004FF40072164900F00DF904F13800009426
:10100000144B15494FF4007200F086F9134BE36559
:101010000B215220256603B0BDE8304000F088B8AF
:101020009C29022080F93703E02A0220050E0008DF
:10103000E030022000440040082A0220E02C022078
:10104000150E0008E032022000480040742A0220F9
:10105000E02E0220250E0008E03402200078004037
:101060002E4B002908BF1946037C8166012B30B541
:101070000CD12B4B984235D12A4B1A6C42F40032DA
:101080001A641A6E42F400321A661B6E0A68036E06
:10109000C46D03EB5203B3FBF2F34A68150442BF7D
:1010A00023F0070503F0070343EA4503E3608B6879
:1010B00043F040036360CB6843F00103A36042F454
:1010C000967343F00103236051054FF0FF33236211
:1010D00005D512F010221DD0B2F1805F1CD080F82F
:1010E000643030BD104B984208D10E4B1A6C42F45C
:1010F00080221A641A6E42F48022C5E70B4B984294
:10110000C4D1084B1A6C42F080421A641A6E42F045
:101110008042B9E77F23E2E73F23E0E7A83A0008EF
:101120009C29022000380240082A0220742A02204A
:1011300000F1604300F01F02400903F5614309011B
:101140008000C9B200F1604083F8001300F56140EF
:1011500001239340C0F8803103607047F8B515460D
:1011600082680669AA420B46816938BF8568761A8B
:10117000B542044607D218462A46FFF7A1FDA369E7
:101180002B44A3610DE011D932461846FFF798FDB4
:10119000AF1B3A46E1683044FFF792FDE2683A44FB
:1011A000A261A3685B1BA3602846F8BD18462A46C7
:1011B000FFF786FDE368E4E783682DE9F041044624
:1011C00093421546266938BF85684069361AB5428C
:1011D0000F4606D22A46FFF773FD63692B4463610D
:1011E0000DE012D93246A5EB0608FFF769FD42462D
:1011F000B919E068FFF764FDE26842446261A368E0
:101200005B1BA3602846BDE8F0812A46FFF758FD26
:10121000E368E4E710B50A440024C361029B006060
:1012200040608460C160816141610261036210BD00
:1012300008B582694369934201D1826882B98268A4
:10124000013282605A1C42611970426903699A42F4
:1012500001D3C3684361002100F098FE002008BD5F
:101260004FF0FF3008BD000070B5202304460E4645
:1012700083F31188A568A5B1A368A269013BA360A7
:10128000531CA36115782269934224BFE368A361CC
:10129000E3690BB120469847002383F31188284661
:1012A00070BD3146204600F061FE0028E2DA85F389
:1012B000118870BD2DE9F74F05460F4690469A46B6
:1012C000D0F81C90202686F311884FF0000B1446AE
:1012D00064B1224639462846FFF740FF034668B905
:1012E0005146284600F042FE0028F1D0002383F347
:1012F0001188A8EB040003B0BDE8F08FB9F1000F2E
:1013000003D001902846C847019B8BF31188E41A4B
:101310001F4486F31188DBE7C16081614161C361CD
:101320001144009B0060406082600161036270476D
:10133000F8B504460E461746202383F31188A568A6
:10134000A5B1A368013BA36063695A1C62611E706A
:10135000236962699A4224BFE3686361E3690BB160
:1013600020469847002080F31188F8BD3946204672
:1013700000F0FCFD0028E2DA85F31188F8BD0000DA
:10138000836942699A4210B501D182687AB982684C
:10139000013282605A1C82611C7803699A4201D32F
:1013A000C3688361002100F0F1FD204610BD4FF0BD
:1013B000FF3010BD2DE9F74F05460F4690469A467F
:1013C000D0F81C90202686F311884FF0000B1446AD
:1013D00064B1224639462846FFF7EEFE034668B957
:1013E0005146284600F0C2FD0028F1D0002383F3C7
:1013F0001188A8EB040003B0BDE8F08FB9F1000F2D
:1014000003D001902846C847019B8BF31188E41A4A
:101410001F4486F31188DBE70268436811430160CB
:1014200003B11847704700001430FFF743BF0000B6
:101430004FF0FF331430FFF73DBF00003830FFF7A7
:10144000B9BF00004FF0FF333830FFF7B3BF0000E3
:101450001430FFF709BF00004FF0FF311430FFF7E1
:1014600003BF00003830FFF763BF00004FF0FF32CA
:101470003830FFF75DBF000000207047FFF774BDF4
:10148000044B0360002343608360C3600123037443
:10149000704700BFC03A000810B52023044683F30C
:1014A0001188FFF7DDFD02232374002383F31188E5
:1014B00010BD000038B5C36904460D461BB90421B0
:1014C0000844FFF7A9FF294604F11400FFF7B0FE16
:1014D000002806DA201D4FF48061BDE83840FFF790
:1014E0009BBF38BD026843681143016003B11847D0
:1014F0007047000013B5446BD4F894341A6811781F
:10150000042916D1217C022913D1197912890123CA
:101510008B4013420DD101A904F14C0001F076FE7D
:10152000024630B1D4F89444019B2179206800F040
:10153000DBF902B010BD0000143001F0E5BD000081
:101540004FF0FF33143001F0DFBD00004C3001F0EC
:10155000C9BE00004FF0FF334C3001F0C3BE0000A5
:10156000143001F0B3BD00004FF0FF31143001F032
:10157000ADBD00004C3001F095BE00004FF0FF32D1
:101580004C3001F08FBE0000D0F8942438B51368B9
:1015900019780429054601D0012038BD017C0229B3
:1015A000FAD112795C89012090400440F4D105F110
:1015B000140001F045FD02460028EDD0D5F8945402
:1015C0004FF480732868697900F07CF9204638BDB3
:1015D000406BFFF7D9BF0000002070477047000044
:1015E0007FB5124B0360002343608360C360012515
:1015F00002260F4B057404460290019300F1840209
:10160000294600964FF48073143001F0F5FC094B25
:101610000193029400964FF4807304F523722946D7
:1016200004F14C0001F0CEFD04B070BDE83A0008B2
:10163000D1150008F51400080B68202282F31188E8
:101640000A7903EB820210624A790D3243F82200D4
:101650008A7912B103EB8203186202230374C0F883
:101660009414002383F311887047000038B50446B2
:10167000012502210430FFF735FF04F1140025771E
:101680006FF0010100F08EFC84F8545004F14C001E
:101690006FF00101BDE8384000F084BC10B50121B5
:1016A00004460430FFF71EFF0023237784F85430EC
:1016B00010BD000038B504460025143001F0B4FC1C
:1016C00004F14C00257701F095FD201D84F854505D
:1016D0000121FFF707FF2046BDE83840FFF754BF60
:1016E00090F85C3003F06003202B19D190F85D2056
:1016F000212A0AD0222A4FF000030ED0202A0FD12F
:10170000084A02650722426504E0064B0365072389
:101710004365002383650120704703654365F9E74E
:101720000020704728240220D0F8943437B51A6876
:101730001178042904461AD1017C022917D119799C
:10174000128901238B40134211D100F14C05284628
:1017500001F026FE58B101A9284601F057FDD4F842
:101760009444019B21790246206800F0BDF803B043
:1017700030BD000000EB8103F7B51C6A05460E463C
:10178000F4B1202383F3118805EB8607201D08217F
:10179000FFF7A8FEFB685B691B684C3413B1204659
:1017A00001F042FD01A9204601F030FD024648B19A
:1017B000019B3146284600F097F8002383F31188F7
:1017C00003B0F0BDFB685A691268002AF5D01B8A85
:1017D000013B1340F1D105F15C02EAE70D3138B568
:1017E00050F82140DCB1202383F31188D4F89424ED
:1017F0001368527903EB8203DB689B695D6845B12E
:1018000004216018FFF76EFE294604F1140001F070
:1018100021FC2046FFF7B8FE002383F3118838BD72
:101820007047000000F0D2BF012303700023436023
:1018300000F1240200F1380142F8043B8A421361AE
:10184000FAD103814381704738B50446202383F3DE
:10185000118800254160C560056145618561C561EC
:10186000056200F0C3FF0223237085F3118838BDA1
:1018700070B500EB810305465069DA600E461446E8
:1018800018B110220021FFF745FAA06918B1102203
:101890000021FFF73FFA31462846BDE8704001F0CD
:1018A0006BB80000028902F001020281428902F055
:1018B000010242810022026142618261C2610262D0
:1018C00001F0EEB8F0B400EB81044789E46801252B
:1018D000A4698D403D43458123600023A26063607D
:1018E000F0BC01F009B90000F0B400EB81040789F5
:1018F000E468012564698D403D4305812360002330
:10190000A2606360F0BC01F083B9000070B50223EF
:10191000002504460370A0F8645080F8665080F8F3
:10192000675005814581C560056145618561C56177
:10193000056280F84C5000F0BBFF63681B6823B160
:1019400029462046BDE87040184770BD43680278BC
:101950001B6880F86820052202700BB1042118472B
:1019600070470000436890F868201B6802700BB154
:10197000052118477047000090F84C3070B50446B8
:1019800013B1002380F84C3004F15C02204601F0D2
:10199000A9F863689B6863BB94F85C5015F0600617
:1019A00015D194F85D3005F07F0545EA032540F236
:1019B00002339D4200F00E815BD8022D00F0DC80E6
:1019C0003FD8002D00F08780012D00F0CF8000214E
:1019D000204601F0F3FA0021204601F0E5FA6368A1
:1019E0001B6813B1062120469847062384F84C3023
:1019F00070BD204698470028CED094F8632094F814
:101A0000623043EA0223626D934238BF636594F902
:101A10005C30656D002B4FF0200380F2FD80002DBF
:101A200000F0EC80092284F84C2083F31188002117
:101A3000636D226D2046FFF757FF002383F3118863
:101A400070BDB5F5817F00F0B180B5F5407F49D01C
:101A5000B5F5807FBBD194F85E30012BB7D1B4F8D7
:101A6000643023F00203A4F8643026656665A66539
:101A7000C3E740F201639D421ED8B5F5C06F3BD26B
:101A8000B5F5A06FA3D1B4F85C30B3F5A06F0ED15B
:101A900094F85E3084F86630204600F061FF636899
:101AA0001B6813B1012120469847032323700023AC
:101AB00023656365A365A0E7B5F5106F32D040F6E6
:101AC00002439D4252D0B5F5006F80D104F1670307
:101AD0002365012324E004F1640323650223636585
:101AE000A5658AE794F85E30012B7FF470AFB4F8F7
:101AF000643043F00203B6E794F86120616894F81B
:101B000060304D6894F85F1043EA0223204694F851
:101B10005E20A84700283FF45AAF43682365036856
:101B20006365A4E72378042B10D1202383F3118865
:101B30002046FFF7B7FE86F31188636884F8676074
:101B40001B68032121700BB12046984794F85E3042
:101B5000002BACD084F867300423237063681B68C3
:101B6000002BA4D0022120469847A0E7374B2365DD
:101B70000223636500239DE794F8601011F0800F45
:101B8000204601F00F010ED000F09EFF012806D084
:101B900002287FF41CAF2E4B2365606567E72D4B51
:101BA0002365656563E700F081FFEFE794F85E3039
:101BB000002B7FF40CAF94F8603013F00F013FF46A
:101BC00076AF1A06204602D501F00CFA6FE701F055
:101BD000FFF96CE794F85E30002B7FF4F8AE94F8D0
:101BE000603013F00F013FF462AF1B06204602D5B0
:101BF00001F0E4F95BE701F0D7F958E7142284F823
:101C00004C2083F311882B462A4629462046FFF7AD
:101C100059FE85F3118870BD5DB1152284F84C2002
:101C200083F311880021636D226D2046FFF74AFE81
:101C300003E70B2284F84C2083F311882B462A46B5
:101C400029462046FFF750FEE3E700BF183B000897
:101C5000103B0008143B000838B590F84C3004469F
:101C6000152B29D8DFE803F03E28282828283E280D
:101C7000280B293928282828282828283E3E90F88B
:101C8000631090F86220436D42EA01229A4214D90F
:101C9000C268128AB3FBF2F502FB15356DB9202339
:101CA00083F311882B462A462946FFF71DFE85F34C
:101CB00011880A2384F84C3038BD142384F84C3042
:101CC000202383F3118800231A4619462046FFF784
:101CD000F9FD002383F3118838BD836D03B1984764
:101CE0000023E7E7002101F069F90021204601F017
:101CF0005BF963681B6813B10621204698470623E9
:101D0000D8E7000090F84C20152A38B5044622D8B0
:101D10000123934040F6416213421DD113F4801514
:101D20000FD19B0217D50B2380F84C30202383F36F
:101D300011882B462A462946FFF7D6FD85F31188E0
:101D400038BDC3689B695B682BB9836D03B1984745
:101D5000002384F84C3038BD002101F02FF9002118
:101D6000204601F021F963681B6813B10621204663
:101D700098470623EDE70000024B00221B605B60E2
:101D80009A607047E0360220002303748268054B96
:101D90001B6899689142FBD25A68036042601060E8
:101DA00058607047E036022008B5202383F311887D
:101DB000037C032B05D0042B0DD02BB983F31188A2
:101DC00008BD436900221A604FF0FF334361FFF7FB
:101DD000DBFF0023F2E790E80C001A600268536012
:101DE000F2E70000002303748268054B1B689968C2
:101DF0009142FBD85A680360426010605860704797
:101E0000E0360220054B19690874186802681A60E8
:101E10005360186101230374FEF786BAE03602208E
:101E200030B54B1C87B005460A4C10D023690A4ACE
:101E300001A800F0D3F82846FFF7E4FF049B13B194
:101E400001A800F007F92369586907B030BDFFF712
:101E5000D9FFF8E7E0360220A91D000838B50C4D7F
:101E600041612B6981689A689142044603D8BDE8B4
:101E70003840FFF789BF1846FFF786FF01232C6122
:101E8000014623742046BDE83840FEF74DBA00BF36
:101E9000E0360220044B1A681B6990689B689842E0
:101EA00094BF002001207047E036022010B5084C96
:101EB000236820691A6822605460012223611A7421
:101EC000FFF790FF01462069BDE81040FEF72CBAED
:101ED000E0360220826002220274002242747047BF
:101EE0008368A3F17C0243F80C2C026943F83C2C74
:101EF000426943F8382C074A43F81C2CC26843F85F
:101F0000102C022203F8082C002203F8072CA3F15E
:101F1000180070474103000810B5202383F311888F
:101F2000FFF7DEFF00210446FFF798FF002383F34D
:101F30001188204610BD0000024B1B6958610F201C
:101F4000FFF760BFE0360220202383F31188FFF7FC
:101F5000F3BF000008B50146202383F31188082051
:101F6000FFF75EFF002383F3118808BD49B1064BDC
:101F700042681B6918605A60136043600420FFF7D1
:101F80004FBF4FF0FF307047E036022003689842A1
:101F900006D01A680260506059611846FFF7F4BE17
:101FA0007047000038B504460D462068844200D1D1
:101FB00038BD036823605C604561FFF7E5FEF4E728
:101FC000054B03F114025A619A614FF0FF32DA6156
:101FD00000221A62704700BFE0360220F8B50361A4
:101FE0004FF08043C2605C6A194B1A46022952F8CE
:101FF000145F38BF0221954206461F460AD1586138
:1020000098611C620560456081600819BDE8F84070
:1020100001F0E8B9186AAB68241A0C1902D3E41A63
:102020002D6804E09C4202D2204401F0E9F9AB683B
:102030009C42F4D86B68736035601E606E60B4605B
:10204000A9684FF0FF33091BA960FB61F8BD00BF11
:10205000E036022010B41B4C234653F8141F814273
:1020600010D0416802680A60026851609A424FF0DD
:102070000001C16003D0936881680B4493605DF8F0
:10208000044B70470A68626100209A425360C8603E
:1020900003D15DF8044B01F0ADB99368886803443F
:1020A00093604FF08042206A526A121A9342E6D936
:1020B000991A012998BF931C18445DF8044B01F04C
:1020C0009FB900BFE036022000207047FEE7000005
:1020D000704700004FF0FF3070470000022906D023
:1020E000032906D00129064818BF0020704705487B
:1020F0007047032A9ABF044800EBC20000207047D3
:10210000083C0008BC3B00083024022070B504469F
:1021100008460D46FEF7F6FDC6B2204601340378A8
:102120000BB9184670BD32462946FEF7D3FD00288C
:10213000F3D1012070BD00002DE9F04F81469BB026
:1021400008460C461646FEF7DDFD3C49C5B2204662
:10215000FFF7DCFF08B10335EDB239492046FFF740
:10216000D5FF08B11035EDB2632D01AF0CD8DFF803
:10217000DCA0DFF8DCB03D4694F80080B8F1000F39
:102180001CD185F8008003E02146384601F05EFC52
:102190003846FEF7B7FDC0B2431C5B0089E8480033
:1021A000337003237370002302361946DAB290426B
:1021B00006F102063AD81BB0BDE8F08FB8F1250F42
:1021C0002FD107221D492046FEF784FD58B9DBF8C0
:1021D00000202A60DBF804206A60BBF808202A810E
:1021E00007340A35C8E7082215492046FEF772FD74
:1021F000B8B91448AA1C10F8011F134B4FEA111E5E
:1022000001F00F011EF80AE011F80A1002F802ECC2
:10221000984202F8011C02F10202ECD11835083490
:10222000AAE785F8008001340135A5E7FA5C06F8D5
:10223000022C06F8011C0133B8E700BF6C3B000814
:10224000743B00081FF4F01F2BF4F01F883B0008BC
:102250007D3B000808B5202383F311880348FFF76E
:1022600063FA002383F3118808BD00BF20370220E2
:1022700010B50446052916D8DFE801F01615031637
:10228000161D202383F311880E4A0121FFF7F0FA6F
:1022900020460D4A0221FFF7EBFA0C48FFF70AFA35
:1022A000002383F3118810BD202383F3118807488E
:1022B000FFF7DCF9F4E7202383F311880348FFF7E5
:1022C000EDF9EDE71C3B0008403B000820370220F9
:1022D00038B50C4D0C4C0D492A4604F10800FFF7A7
:1022E0002BFF05F1CA0204F110000949FFF724FF92
:1022F00005F5CA7204F118000649BDE83840FFF739
:102300001BBF00BFE83B0220302402209C3B00089A
:10231000A03B0008743B0008BFF34F8F024AD3680C
:10232000DB03FCD4704700BF003C024008B5074BFC
:102330001B7853B9FFF7F0FF054B1A69002ABFBF9E
:10234000044A5A6002F188325A6008BD463E0220B3
:10235000003C02402301674508B5054B1B7833B9A3
:10236000FFF7DAFF034A136943F00043136108BD26
:10237000463E0220003C02400B2870B513D80B4AA1
:102380000B4C137863B90B4E4FF0006144F82310E7
:1023900056F8235001330C2B2944F7D10123137035
:1023A00054F8200070BD002070BD00BF783E0220B0
:1023B000483E0220283C0008014B53F8200070479B
:1023C000283C00080C2070470B2810B5044601D9A2
:1023D000002010BDFFF7D0FF064B53F824301844FF
:1023E000C21A0BB9012010BD12680132F0D1043BB2
:1023F000F6E700BF283C00080B2810B504462FD88C
:10240000FFF78AFFFFF792FF1649F323CB60FFF730
:1024100083FFC300DBB243F4007343F002030B619C
:102420000B6943F480330B61FFF776FFFFF7A4FFDE
:102430000D4B53F824300344BFF34F8F0B4A98429F
:102440000AD3BFF34F8FBFF36F8FFFF785FF20468F
:10245000BDE81040FFF7B8BFC2F85C022030EEE7DD
:10246000002010BD003C0240283C000800ED00E0C8
:102470002DE9F047D40715464DD41318B3F1026F78
:1024800049D2324B1B68DA0745D5314CFFF74EFF76
:10249000F323E360FFF740FF2F46401A40F2012983
:1024A000032F884601EB000618D8294C40F2011989
:1024B0007B1A4344012B01EB000623692FD823F03C
:1024C00001032361FFF748FF2846BDE8F08736681F
:1024D00051F8043CB34218D1043FE1E7B307E4D11B
:1024E000236923F440732361236943EA09032361C9
:1024F0000431D8F800303360BFF34F8FFFF70CFF83
:10250000E368002BE3D0F323E360236923F00103A6
:102510002361FFF721FF4FF0FF30BDE8F08723F480
:1025200040732361236943EA090323618A4631F832
:10253000023B3380BFF34F8FFFF7EEFE3688BAF8C9
:102540000030B6B2B342B3D0DFE700BF003802407C
:10255000003C0240084908B50B7828B153B9FFF791
:10256000E5FE01230B7008BD23B1BDE808400870EB
:10257000FFF7F2BE08BD00BF463E0220014B186DBA
:10258000704700BF00280040094B1A6F120407D49F
:102590001A6F42F400721A671A6F42F400421A6707
:1025A000044A136843F480731360034B1865704743
:1025B000003802400070004000280040064A53687E
:1025C00023F001035360EFF30983683383F3098831
:1025D000002383F31188704730EF00E010B520230B
:1025E00083F31188104B5B6813F4006318D0F1EE8D
:1025F000103AEFF309844FF0807344F84C3C0B4BD6
:10260000DB6844F8083CA4F1680383F30988FFF70A
:1026100041FC18B1064B44F8503C10BD054BFAE79D
:1026200083F3118810BD00BF00ED00E030EF00E043
:102630005103000854030008F0B5BFF34F8FBFF3F8
:102640006F8F1D4B0021C3F85012BFF34F8FBFF3A4
:102650006F8F5A6942F400325A61BFF34F8FBFF354
:102660006F8FC3F88410BFF34F8FD3F88020C2F36D
:10267000C904C2F34E325201A50743F6E07602EADE
:10268000060E284621464EEA00070139C3F860725B
:102690004F1C00F14040F6D1203A12F1200FEED14C
:1026A000BFF34F8F5A6942F480325A61BFF34F8FA4
:1026B000BFF36F8FF0BD00BF00ED00E0FEE700004C
:1026C000084A094B09498B4204D3094A0021934225
:1026D00005D3704752F8040F43F8040BF3E743F8AF
:1026E000041BF4E7343E00088841022088410220A0
:1026F00088410220036F30B500229D68C46E1146E8
:102700004FF0FF3004EB421301329542C3F8001939
:10271000C3F81019C3F80809C3F8001BC3F8101B4D
:10272000C3F8080BEED24FF00113C4F81C3830BDCB
:10273000890141F02001016103699B06FCD412204C
:1027400000F0ECBE204B03EB80022DE9F047D2F8FD
:102750000CE0DD6EDEF81420461CD2F800C005EB5C
:10276000063605EB4018516861450BD3D5F834287F
:10277000012303FA00F022EA0000C5F834081846E5
:10278000BDE8F087BEF81040ACEB0103A34228BFC0
:102790002346D8F81849A4B2B3EB840F10D8946834
:1027A0001F46A4F1040959F804AFC6F800A0042F8D
:1027B00001D9043FF7E71C440B4494605360D2E70F
:1027C0000020BDE8F08700BF7C3E022010B5054C1C
:1027D0002046FFF729F84FF0A043E366024B23673A
:1027E00010BD00BF7C3E02207C3C00080378012B1A
:1027F00070B505464DD1284BC46E98421BD1274B6E
:102800005A6B42F080025A635A6D42F080025A6558
:102810005A6D5A6942F080025A615A6922F0800268
:102820005A610E2143205B69FEF782FC1C4BE3607A
:102830001C4BC4F800380023C4F8003EC0232360BA
:102840004FF40413A363EE6E202000F067FE012313
:1028500033613369DB07FCD4122000F05FFE33697B
:10286000002BFCDA0026A6602846FFF743FF6B68C2
:10287000C4F81068DB68C4F81468C4F81C684BB965
:10288000094BA3614FF0FF336361A36843F0010379
:10289000A36070BD054BF4E77C3E02200038024087
:1028A0004014004003002002003C30C0083C30C00F
:1028B000F8B5C46E054600212046FFF739FF296FA1
:1028C00000234FF001128F68C4F834384FF00066CF
:1028D000C4F81C284FF0FF3004EB431201339F4231
:1028E000C2F80069C2F8006BC2F80809C2F8080B08
:1028F000F2D20B68EA6E6B6763621023136116698C
:1029000016F01006FBD1122000F008FED4F80038B3
:1029100023F4FE63C4F80038A36943F4402343F072
:102920001003A3610923C4F81038C4F814380A4B03
:10293000EB604FF0C043C4F8103B084BC4F8003BB9
:10294000C4F81069C4F800396B6F03F1100243F446
:1029500080136A67A362F8BD583C000840800010ED
:10296000C26E90F86610D2F8003823F4FE6343EA92
:102970000113C2F8003870472DE9F0410EB200EBA8
:1029800086080D46D8F80C100F6807F00303022BD9
:1029900050D0032B50D03D4A3D4F012B18BF174656
:1029A000C46E4FEA451E04EB0E030022C3F8102B41
:1029B0008A6905F1100C002A40D04A8A05F15803B3
:1029C0005B013A43E2500123D4F81C2803FA0CF3CC
:1029D0001343A6444A69C4F81C380023CEF81039C2
:1029E00005F13F03002A39D00A8A898B9208012910
:1029F00088BF4A43416F04EB8303561841EA024201
:102A0000466729465A602046FFF792FED8F80C30F8
:102A10001B8A43EA85531F4305F148035B01E750D6
:102A20000123D4F81C2803FA05F51543C4F81C58F3
:102A3000BDE8F081174FB3E7174FB1E704EB46133A
:102A4000D3F8002B22F40042C3F8002BD4F81C2842
:102A5000012303FA0CF322EA0303BAE704EB83032E
:102A60000E4A5A6004EB461629462046FFF760FEE0
:102A7000D6F8003923F40043C6F80039D4F81C38DE
:102A8000012202FA05F523EA0505CFE700800010D0
:102A9000008004100080081000800C100004000268
:102AA000026F12684267FFF725BE00005831C36EFF
:102AB00049015B5813F4004004D013F4001F14BF05
:102AC00001200220704700004831C36E49015B5865
:102AD00013F4004004D013F4001F14BF012002209F
:102AE0007047000000EB8101CB68196A0B68136026
:102AF0004B6853607047000000EB810330B5DD6820
:102B0000AA691368D36019B9402B84BF40231360AE
:102B10006B8A1468C26E1C44013CB4FBF3F463433B
:102B2000033323F0030302EB411043EAC44343F0B1
:102B3000C043C0F8103B2B6803F00303012B09B21C
:102B40000ED1D2F8083802EB411013F4807FD0F890
:102B5000003B14BF43F0805343F00053C0F8003BE8
:102B600002EB4112D2F8003B43F00443C2F8003BB1
:102B700030BD00002DE9F041244DEE6E06EB401310
:102B80000446D3F8087BC3F8087B38070AD5D6F883
:102B90001438190706D505EB84032146DB6828465F
:102BA0005B689847FA072FD5D6F81438DB072BD582
:102BB00005EB8403D968CCB98B69488A5E68B6FB9B
:102BC000F0F200FB12628AB91868DA6890420DD2FE
:102BD000121A83E81400202383F311880B4821463E
:102BE000FFF78AFF84F31188BDE8F081012303FA1F
:102BF00004F26B8923EA02036B81CB6823B121467F
:102C00000248BDE8F0411847BDE8F0817C3E022053
:102C100000EB810370B5DD68C36E6C692668E66001
:102C20004A0156BB1A444FF40020C2F810092A6822
:102C300002F00302012A0AB20ED1D3F8080803EB0E
:102C4000421410F4807FD4F8000914BF40F0805083
:102C500040F00050C4F8000903EB4212D2F800091A
:102C600040F00440C2F80009D3F83408012202FA07
:102C700001F10143C3F8341870BD19B9402E84BF67
:102C80004020206020682E8A841940F00050013CCA
:102C90001A44B4FBF6F440EAC440C6E7F8B504466B
:102CA0001E48C56E05EB4413D3F80869C3F80869DC
:102CB000F10717D5D5F81038DA0713D500EB8403E0
:102CC000D9684B691F68DA68974218D2D21B00276F
:102CD0001A605F60202383F311882146FFF798FF75
:102CE00087F31188330617D5D5F834280123A3407C
:102CF000134211D02046BDE8F840FFF723BD012361
:102D000003FA04F2038923EA020303818B68002B90
:102D1000E8D021469847E5E7F8BD00BF7C3E022099
:102D2000A0482DE9F84FC56E6E69AB691E4016F4D8
:102D3000805F6E61044605D0FEF7E8FDBDE8F84F00
:102D4000FFF74CBC002E12DAD5F8003E95489B07E1
:102D50001EBFD5F8003E23F00303C5F8003ED5F8AA
:102D6000043823F00103C5F80438FEF7FBFD3705EE
:102D700002D58C48FEF7EAFDB0040CD5D5F808382A
:102D800013F0060FEB6823F470530CBF43F4105399
:102D900043F4A053EB60310704D56368DB680BB1E3
:102DA00080489847F2026FD4B3020CD5D4F86C80F7
:102DB000DFF8F0A100274FF00109236F9B68F9B2FB
:102DC0008B4280F09C80F70619D5E16E0A6AC2F347
:102DD0000A1702F00F0302F4F012B2F5802F00F090
:102DE000B680B2F5402F0AD104EB830301F5805180
:102DF000DB68186A00231A469F4240F09C80330328
:102E0000D5F818481DD5E70302D50020FFF7B2FE1C
:102E1000A50302D50120FFF7ADFE600302D5022015
:102E2000FFF7A8FE210302D50320FFF7A3FEE2026D
:102E300002D50420FFF79EFEA30202D50520FFF76E
:102E400099FE77037FF57AAFE60702D50020FFF7FA
:102E500025FFA50702D50120FFF720FF600702D557
:102E60000220FFF71BFF210702D50320FFF716FF03
:102E7000E20602D50420FFF711FFA3067FF55EAF3F
:102E80000520FFF70BFF59E7D4F86C80DFF814A199
:102E900000274FF00109236F9B685FFA87FB5B45B2
:102EA00082D308EB4B13D3F8002902F44022B2F589
:102EB000802F22D1D3F80029002A1EDAD3F8002966
:102EC00042F09042C3F80029D3F80029002AFBDB26
:102ED0005946E06EFFF72CFC228909FA0BF322EA2F
:102EE0000303238104EB8B03DB689B6813B1594612
:102EF000504698475846FFF725FC0137CBE708EBCB
:102F00004112D2F8003B03F44023B3F5802F10D1D7
:102F1000D2F8003B002B0CDA628909FA01F322EAAD
:102F20000303638104EB8103DB68DB680BB150466C
:102F30009847013741E79C0708BF0A68072B98BFED
:102F4000027003F101039CBF120A013054E70233FF
:102F500004EB830201F58051526890690268D0F851
:102F600008C04068A2EB000E0022104697420AD12A
:102F700004EB830463689B699A683A449A605A68D0
:102F800017445F603BE712F0030F08BF08689645DF
:102F900088BF8CF8000002F1010284BF000A0CF126
:102FA000010CE3E77C3E0220C36E03EB4111D1F834
:102FB000003B43F40013C1F8003B7047C36E03EBC2
:102FC0004111D1F8003943F40013C1F800397047BA
:102FD000C36E03EB4111D1F8003B23F40013C1F899
:102FE000003B7047C36E03EB4111D1F8003923F465
:102FF0000013C1F80039704730B5039C01720433E7
:1030000004FB0325C361049B03630021059B00604F
:103010004060C16042610261856104624262816216
:10302000C162436330BD00000022416A4161016119
:10303000C2608262C2626FF00101FEF7B3BF00009E
:1030400003694269934203D1C2680AB10020704704
:10305000181D704703691960C2680132C260C269F5
:10306000134482690361934224BF436A03610021D0
:10307000FEF78CBF38B504460D46E3683BB1626984
:10308000131D1268A3621344E362002038BD237A43
:1030900033B929462046FEF769FF0028EDDA38BD2E
:1030A0006FF00100FBE70000C368C269013BC36029
:1030B0004369134482694361934224BF436A436175
:1030C00000238362036B03B11847704770B5202358
:1030D000044683F31188866A3EB9FFF7CBFF0546A5
:1030E00018B186F31188284670BDA36AE26A13F806
:1030F000015BA362934202D32046FFF7D5FF002372
:1031000083F31188EFE700002DE9F74F1F460446CF
:103110000E469146202383F311884FF08048002506
:10312000D8F82430FB18009307F1FF3AAB46A36AA6
:10313000ABB91AF1030F06D939462046FFF79AFFBB
:1031400068B1002305E0D8F82410009A511A8F4284
:10315000F3D283F31188284603B0BDE8F08FA16A4B
:10316000E36AA9EB05025B1A934228BF1346402B82
:103170001CD9334601F1400251F8040B43F8040B0B
:103180009142F9D1A36A40334036A3624035A26A26
:10319000E36A9A4202D32046FFF786FF8BF3118839
:1031A0004D45D8D2202383F31188C0E71A46304614
:1031B0000193FDF785FD019BA26A1A441E44A26299
:1031C0001D44E4E710B5029C0172043303FB0421A3
:1031D000C36100238362C362039B0363049B00609B
:1031E0004060C46042610261816104624262436383
:1031F00010BD0000026AC260426A426102610022A0
:103200008262C2626FF00101FEF7CCBE43690269BF
:103210009A4203D1C2680AB100207047184650F89C
:10322000043B0B6070470000C368C2690133C36090
:103230004369134482694361934224BF436A4361F3
:103240000021FEF7A3BE000038B504460D46E36832
:103250003BB123691A1DA262E2691344E3620020B4
:1032600038BD237A33B929462046FEF77FFE002871
:10327000EDDA38BD6FF00100FBE70000036919606B
:10328000C268013AC260C269134482690361934211
:1032900024BF436A036100238362036B03B11847B1
:1032A0007047000070B5202304460E4683F3118852
:1032B000856A35B91146FFF7C7FF10B185F311884C
:1032C00070BDA36A1E70A36AE26A01339342A362CF
:1032D00004D3E16920460439FFF7D0FF002080F3D2
:1032E000118870BD2DE9F74F1F4604460D469146E3
:1032F000202383F311884FF080480026D8F824302B
:10330000FB18009307F1FF3AB346A36AABB91AF171
:10331000030F06D939462046FFF796FF68B1002310
:1033200005E0D8F82410009A511A8F42F3D283F3A3
:103330001188304603B0BDE8F08FA06AE36AA9EBBC
:1033400006021B1A934228BF1346402B1CD905F1D5
:10335000400355F8042B40F8042B9D42F9D1A36A91
:103360004033A3624036A26AE36A9A4204D3E16919
:1033700020460439FFF782FF8BF311884E45D8D2DF
:10338000202383F31188C0E71A4629460193FDF7ED
:1033900097FC019BA26A1A441D44A2621E44E2E704
:1033A000026943699A4203D1C3681BB91846704742
:1033B0000023FBE7836A002BF8D0043B9B1AF5D06F
:1033C0001360C368013BC360C3691A448369026127
:1033D0009A4224BF436A0361002383620123E5E725
:1033E00000F040B94FF08043002258631A61022276
:1033F000DA6070474FF080430022DA6070470000C7
:103400004FF0804358637047FEE7000010B5194C39
:10341000FEF7B2FCFEF7D4FD802217492046FEF7E6
:1034200059FD012344F8180C0374144B144AD9684D
:1034300021F4E0610904090C0A431249DA60CA6800
:1034400042F08072CA60104A1049C2F8B01F116879
:1034500041F0010111601022DA77202283F8222046
:10346000002383F3118862B60948BDE81040FEF7D7
:1034700053BD00BF08370220883C000800ED00E083
:103480000003FA05F0ED00E0001000E055CEACC5F9
:10349000903C00082DE9F84F1F4C4FF0000865697B
:1034A00004F11407C1464FF08043266A5B6AAA689C
:1034B0009E1B96421DD34FF0200AAA68236AD5F8B6
:1034C0000CB0134423622B68BB425F60A6EB02067C
:1034D0006361C5F80C8001D1FFF78CFF89F3118877
:1034E0002869D8478AF311886569AB689E42E4D29F
:1034F000D9E76269BA420CD0916823628E1B96604C
:10350000A86802282CBF1818981CBDE8F84FFFF7D0
:1035100077BFBDE8F88F00BFE0360220034B596843
:103520005A68521A9042FBD8704700BF001000E062
:103530004B6843608B688360CB68C3600B694361F1
:103540004B6903628B6943620B680360704700003C
:1035500008B5274B27481A6940F2FF710A431A61E0
:103560001A6922F4FF6222F007021A611A691A6BC3
:103570000A431A631A6D0A431A651F4A1B6D1146E6
:10358000FFF7D6FF1D4802F11C01FFF7D1FF1C48D1
:1035900002F13801FFF7CCFF1A4802F15401FFF79E
:1035A000C7FF194802F17001FFF7C2FF174802F187
:1035B0008C01FFF7BDFF164802F1A801FFF7B8FF25
:1035C000144802F1C401FFF7B3FF134802F1E00110
:1035D000FFF7AEFF114802F1FC01FFF7A9FF104809
:1035E00002F58C71FFF7A4FFBDE8084000F09CB81D
:1035F0000038024000000240B03C000800040240D5
:1036000000080240000C024000100240001402407A
:1036100000180240001C024000200240002402402A
:103620000028024008B500F0F3F9FFF7EFFEBDE80F
:103630000840FEF74DBE0000704700004FF0804389
:1036400010B51A69920708D500241C61202383F362
:103650001188FFF71FFF84F31188BDE81040FEF7C3
:10366000BDBF0000104B1A6C42F001021A641A6EC2
:1036700042F001021A660D4A1B6E936843F0010383
:1036800093604FF080436B229A624FF0FF32DA6210
:1036900000229A615A63DA605A6001225A61082155
:1036A0001A601C20FDF744BD00380240002004E0F1
:1036B0001B4B1A696FEA42526FEA52521A611A6939
:1036C000C2F30A021A614FF0FF301A695A69586151
:1036D00000215A6959615A691A6A62F080521A6265
:1036E0001A6A02F080521A621A6A5A6A58625A6A50
:1036F00059625A6A0B4A106840F480701060186F63
:1037000000F44070B0F5007F1EBF4FF480301867A2
:103710001967536823F40073536000F059B900BF70
:103720000038024000700040354B364A1A64364A71
:103730004FF4404111601A6842F001021A601A68A1
:103740009207FCD59A6822F003029A602C4B194626
:103750009A6812F00C02FBD1186800F0F9001860AA
:103760009A601A6842F480321A600B689B03FCD599
:103770004B6F43F001034B67214B5A6F9007FCD509
:10378000224A5A601A6842F080721A601E4B1A462A
:1037900059684904FCD5196841F4803119605368AF
:1037A000D803FCD5136843F400331360164A5368FA
:1037B0009903FCD5124B1A689201FCD5144A9A6001
:1037C00040F20112C3F88C200022C3F89020114A65
:1037D00040F2073111609A6842F002029A60084B89
:1037E0009A6802F00C02082AFAD15A6C42F480421C
:1037F0005A645A6E42F480425A665B6E704700BF4C
:10380000003802400004001000700040186C4009AD
:1038100000948838003C0240084A08B55369116892
:103820000B4003F00103536123B1054A13680BB148
:1038300050689847BDE80840FEF7D0BE003C014004
:1038400008410220084A08B5536911680B4003F08B
:103850000203536123B1054A93680BB1D0689847BE
:10386000BDE80840FEF7BABE003C01400841022016
:10387000084A08B5536911680B4003F0040353610B
:1038800023B1054A13690BB150699847BDE8084058
:10389000FEF7A4BE003C014008410220084A08B5DA
:1038A000536911680B4003F00803536123B1054AC3
:1038B00093690BB1D0699847BDE80840FEF78EBE0A
:1038C000003C014008410220084A08B553691168CC
:1038D0000B4003F01003536123B1054A136A0BB187
:1038E000506A9847BDE80840FEF778BE003C0140AA
:1038F00008410220174B10B55C691A68144004F4A3
:1039000078725A61A30604D5134A936A0BB1D06A40
:103910009847600604D5104A136B0BB1506B98475B
:10392000210604D50C4A936B0BB1D06B9847E20586
:1039300004D5094A136C0BB1506C9847A30504D504
:10394000054A936C0BB1D06C9847BDE81040FEF768
:1039500045BE00BF003C0140084102201A4B10B593
:103960005C691A68144004F47C425A61620504D50B
:10397000164A136D0BB1506D9847230504D5134AB1
:10398000936D0BB1D06D9847E00404D50F4A136EC8
:103990000BB1506E9847A10404D50C4A936E0BB13D
:1039A000D06E9847620404D5084A136F0BB1506F6C
:1039B0009847230404D5054A936F0BB1D06F9847FD
:1039C000BDE81040FEF70ABE003C0140084102205D
:1039D000062108B50846FDF7ABFB06210720FDF7D9
:1039E000A7FB06210820FDF7A3FB06210920FDF710
:1039F0009FFB06210A20FDF79BFB06211720FDF700
:103A000097FB06212820BDE80840FDF791BB000088
:103A100008B5FFF74DFE00F00DF8FDF72FFDFDF79F
:103A200001FFFDF7DBFDFFF707FEBDE80840FFF7EC
:103A3000D7BC0000002304491A465A50C81808335E
:103A4000802B4260F9D1704708410220034611F8EB
:103A5000012B03F8012B002AF9D170471210121321
:103A6000121100000010410001105A0020370220FE
:103A70009C290220082A0220742A022053544D3324
:103A800032463F3F3F3F3F3F0053544D333246376E
:103A90005B347C355D780053544D333246375B36AA
:103AA0007C375D78000000000096000000000000F8
:103AB0000000000000000000000000000000000006
:103AC0000000000045140008311400086D140008BF
:103AD0005914000865140008511400083D1400082A
:103AE000291400087914000800000000551500088A
:103AF000411500087D1500086915000875150008B6
:103B0000611500084D15000839150008D915000881
:103B100000000000010000000000000002000000A2
:103B20000000000075170008DD1700084000400085
:103B3000B83B0220C83B0220020000000000000049
:103B40000300000000000000211800080000000031
:103B500010000000D83B022000000000010000001F
:103B6000000000007C3E02200101020025424F417E
:103B7000524425002553455249414C25006D526F52
:103B80005832312D3737370030313233343536370C
:103B90003839414243444546000000006D526F00F1
:103BA00058322E312D3737370000000071220008BF
:103BB000DD200008E116000855220008430000003F
:103BC000C43B000809024300020100C0320904009E
:103BD000000102020100052400100105240100017A
:103BE000042402020524060001070582030800FFE1
:103BF00009040100020A000000070501024000005C
:103C0000070581024000000012000000103C00087F
:103C1000120110010200004083044057000201021B
:103C2000030100000403090400800000008000007C
:103C3000008000000080000000000200000004007E
:103C40000000040000000400000004000000040064
:103C500000000400000004000000000079190008C2
:103C6000591C0008051D000840004000F43E0220D9
:103C7000F43E022001000000043F0220800000000A
:103C800040010000050000006D61696E0000000049
:103C9000A83C0008103F022008410220010000005B
:103CA000093400080000000069646C650000000031
:103CB0000000802A00000000AAAAAAAA00000000B2
:103CC000FFFF00000000000000A00A00000000004C
:103CD00000000000AAAAAAAA00000000FFFF00003E
:103CE00000000000000000000000000000000000D4
:103CF000AAAAAAAA00000000FFFF0000000000001E
:103D00000000000080298A0100000000AAAAAAAAD7
:103D100040154501FFFF000000707007777000003C
:103D20000080020100000000AAAAAAAA0040010027
:103D3000FFFF0000000000800800000000000000FD
:103D400000000000AAAAAAAA00000000FFFF0000CD
:103D50000000000000000000000000000000000063
:103D6000AAAAAAAA00000000FFFF000000000000AD
:103D7000000000000000000000000000AAAAAAAA9B
:103D800000000000FFFF0000000000000000000035
:103D90000000000000000000AAAAAAAA000000007B
:103DA000FFFF000000000000000000000000000015
:103DB0000000000000000000000000000000000003
:103DC00000000000000000000000000000000000F3
:103DD00000000000000000000000000000000000E3
:103DE0000000000000000000FF00000000000000D4
:103DF0007C3A00083F00000049040000893A0008AE
:103E00003F00000051040000973A00083F00000006
:103E1000009600000000080004000000243C000898
:103E20000000000000000000000000000000000092
:083E300000000000000000008A
:00000001FF
